:03000000022B5A76
:0C2B5A0078FFE4F6D8FD758153022BA132
:100F3F0020000A3C2E2E2E3E004950436F6E6E65E8
:100F4F0063745245510A004950436F6E6E65637466
:100F5F00000A49504E6F41434B210A003E432C5625
:100F6F002C43432CC0E4E0EFF2E5F020D1E8EDEAAA
:100F7F00EEEC49500A003E432C4D41432C253032B4
:100F8F0062583A25303262583A25303262583A2543
:100F9F00303262583A25303262583A253032625830
:100FAF002C4D414320E0E4F0E5F10A003E432C567E
:100FBF0045522C20332E3220EEF22025732025733C
:100FCF002CC2E5F0F1E8FF20495020ECEEE4F3EB02
:100FDF00FF0A004D61722030372032303039003136
:100FEF00303A35393A3431003E432C4C442C505270
:100FFF004F473A2020202020202020202020202072
:10100F0020202020202020202020202020202020D1
:10101F0020202020202020202020202020202020C1
:10102F0020202020202020202020202020202020B1
:10103F0020202020202020202CC4E0F2E020EFF000
:10104F00EEF8E8E2EAE828F4E0E9EB290A003E2AA4
:10105F002C312CCEF1EDEEE2EDFBE520EFE0F0E0F0
:10106F00ECE5F2F0FB20F1E5F2E5E2EEE3EE20E84D
:10107F00EDF2E5F0F4E5E9F1E00A003E412C4130F4
:10108F00312C2562752E2562752E2562752E2562EF
:10109F00752C495020E0E4F0E5F120E0E4E0EFF2B8
:1010AF00E5F0E00A003E412C4130322C2562752ECE
:1010BF002562752E2562752E2562752C495020E00C
:1010CF00E4F0E5F120EEF1ED2E20F1E5F0E2E5F0B0
:1010DF00E00A003E412C4130332C2562752E2562EB
:1010EF00752E2562752E2562752C495020E0E4F08F
:1010FF00E5F120F0E5E72E20F1E5F0E2E5F0E00A7A
:10110F00003E412C4130342C2562752E2562752E00
:10111F002562752E2562752CCCE0F1EAE020F1E511
:10112F00F2E80A003E412C4130352C2562752E2500
:10113F0062752E2562752E2562752CD8EBFEE70A97
:10114F00003E2A2C312CC4EEEF2E20EFE0F0E0EC25
:10115F00E5F2F0FB20F1E5F2E5E2EEE3EE20E8ED5B
:10116F00F2E5F0F4E5E9F1E00A003E422C533031AC
:10117F002C2562752CC6E4E0F2FC20E7E0EFF0EEE0
:10118F00F1E020F1EEE5E4E8EDE5EDE8FF20EEF229
:10119F0020F1E5F0E2E5F0E00A003E422C53303258
:1011AF002C2562752CCEE1ECE5ED20F120F1E5F078
:1011BF00E2E5F0EEEC20E1E5E720EAE2E8F2E0ED2F
:1011CF00F6E8E90A003E422C5330332C2562752C89
:1011DF00CFE5F0E5E7E0EFF3F1EA20EFF0E820EFFD
:1011EF00EEF2E5F0E520F1E2FFE7E820F120F1E58E
:1011FF00F0E2E5F0EEEC0A003E454E440A000A44E8
:10120F00756D705820202020203030203031203054
:10121F0032203033203034203035203036203037F4
:10122F0020303820303920304120304220304320C8
:10123F003044203045203046000A3A003A20000A58
:10124F00000A44756D70442020202020303020305B
:10125F0031203032203033203034203035203036BA
:10126F002030372030382030392030412030422094
:10127F0030432030442030452030460045727220E4
:10128F006B657900526420656570726F6D0A00524C
:10129F0064204D454D0A00526420436F64650A0077
:1012AF00577269746520436F64650A0044656275FF
:1012BF00674950204F4E0A004465627567495020B8
:1012CF004F46460A00446562756755736572204F35
:1012DF006E0A00446562756755736572204F464606
:1012EF000A0044656275674D7367204F6E0A0044AC
:1012FF00656275674D7367204F46460A00436F6EF0
:10130F00666967206C6F636B210A005772206565F1
:10131F0070726F6D0A00205361766520656570727B
:10132F006F6D210A00457272204D414321004C6FB1
:10133F0061643E3E002A00CEF8E8E1EAE00A0020B0
:10134F002D202575282575290A003C4130313D0097
:10135F003C4130323D003C4130333D003C41303464
:10136F003D003C4130353D003C21003C5330313D88
:10137F00003C5330323D003C5330333D003C533042
:09138F00353D003C5330363D00B1
:0633AA00010B0001090007
:1033E000C28E438910758BFF758DB7D2ABD28E22FA
:03001B000229AD0A
:1029AD00C0E0C083C082C0D0C28E758BFF758DB75D
:1029BD0020060675A61E75A6E10509D202E50B6077
:1029CD0002050BE50AD394014002150A050EE50E2A
:1029DD00540F7048D20EE50E543F7012D20090661F
:1029ED008DE0600A04F0E0D394B44002D206906604
:1029FD0086E0600204F0906104E0600214F09066DD
:102A0D008EE0D394014003E014F0300502050CE58F
:102A1D000DD394644004D2068002050DE508D394CD
:102A2D000140021508D28ED0D0D082D083D0E032B2
:1008D000C291C290D2B5C20B7D027C007F07123359
:1008E0008D8F24E524646060097D017F60123328C8
:1008F000D20BE4FDFC7F0B12338D8F24E52430E610
:10090000097D04E4FF12334CD20B7D017C007F078C
:1009100012338D8F24E5247008FD7FFF123328D217
:100920000B300B03126000C288C2A8C2AA758900EE
:10093000122E8290633EE0B4FA06A3E064CE607BA0
:10094000E4F52474362524F582E43463F583E4F079
:100950000524E524B443EC90633E74FAF0A374CE0E
:10096000F0A374CCF0906344740AF0E4A3F0A30401
:10097000F0A3F090633A74FFF0A3F0A3F0E4A3F0C7
:10098000906355740AF0E4F524E5242401FFE43370
:10099000FE74362524F582E43463F583E0FD1233DA
:1009A000040524E524C3944340DFE4F5A775A61E9F
:1009B00075A6E1907FF0F0A3F080FE906349740388
:1009C000F0A374CCF0E4906348F090668BF0A3F051
:1009D0001226CBC2B51231CBC206123118D20BC2CD
:1009E0000DC20C9065767408F09062B47424F0E443
:1009F000A3F090633EE09062B6F090633FE09062B7
:100A0000B7F0906340E09062B8F0906341E090628C
:100A1000B9F0906342E09062BAF0906343E0906274
:100A2000BBF0750A01E4906577F0C207C208C209FD
:100A3000C20A200B18AF24FE7D031225EAE4FF1240
:100A400028FD7E0F7F3FE4FBFDFC1222F790668DB0
:100A5000E060037401F0E4906104F0F50C906575BA
:100A6000F0F50D1233E075A70775A61E75A6E1D245
:100A7000AFE4F50D906104E070031232D590668EFC
:100A8000E06401701D9080007410F09080A874FFE5
:100A9000F0A3F0A3F0A3F0E490668EF0D20BC20CAA
:100AA000C20D908008E0F52430E405D2077410F000
:100AB000E52430E508D2099080087420F0E5243060
:100AC000E608D2089080087440F0E50CC394034017
:100AD00019908002E4F0908001F0908000F0E50C25
:100AE00094064006E4F50C1231189080A0E07003E3
:100AF000122FF19080B8E07003122F009080D0E0A8
:100B000070031230BC908000E07013300710122385
:100B1000FE906331EFF0D3940040031200269080E2
:100B200002E07006908000E06005D205020A71C202
:100B300005E4F50C906104E06003020A71200B12D9
:100B4000906578E0600C7E0F7F41122502E490658D
:100B500078F0300912122186906331EFF0D39400BF
:100B60004005E0FF120022200803020CE7121FFFDD
:100B7000906331EFF07003020A71906375E054BF27
:100B8000247F7003020C50147003020C28240260AE
:100B900003020C89200B077E0F7F48122502200FCD
:100BA00003020CE790634DE07006906351E06067CC
:100BB000906682E0FF90634DE0B50724906683E085
:100BC000FE90634EE0B50618906684E0FE90634F99
:100BD000E0B5060C906685E0FE906350E06E6037ED
:100BE000906351E06F6003020CE7906683E0FF9032
:100BF0006352E06F6003020CE7906684E0FF90634D
:100C000053E06F6003020CE7906685E0FF90635449
:100C1000E06F6003020CE7C2039065777401F01285
:100C20003402750A01020CE790668DE060037401DE
:100C3000F090667AE0FF906377E06F6003020CE764
:100C400090667AE004F0E4F50A906575F0020CE72E
:100C5000300303020CE7906344E07003020A7190D2
:100C60006355740AF01233FBD203E4F50A906575FC
:100C7000F090668604F0E4906679F0A3F0200B67AC
:100C80007E0F7F56122502805E90668DE0600374B1
:100C900001F0300352906375E020E74B906377E0FA
:100CA000FF906679E0FE6F600D906681E07007EE60
:100CB000146F70338013906679E004F0906331E034
:100CC000FFD39404400312284A9060007482F0A37A
:100CD0007401F0906377E0906002F07E607F007DA9
:100CE00003122C6D020A71200303020DFFE50A7046
:100CF00068122A3DEF60237E647F75906476E0245D
:100D000004FD122C6D906681E07009906355E0F54A
:100D10000A020A71E4F50A020A71906686E0D39429
:100D20003C4036906681E0703090668604F0122771
:100D300095E4906475F0A37412F090667AE0906484
:100D400077F0A374FDF090610563A201906479636C
:100D5000A2017F12121D4D809E1233F08F24E524D4
:100D6000B401159060007483F0E4A3F07E607F000E
:100D70007D02122C6D020A71E524D39401401C906F
:100D800060007483F0A37401F0E52424FEA3F07ED8
:100D9000607F007D03122C6D020A71E50A64016018
:100DA00003020A71906575E004F0200B077E0F7F47
:100DB00060122502906355E0C394C85004E02432C9
:100DC000F0906575E0C39405400DC203E49065772B
:100DD000F0123402020A717C667D82906349E0FA67
:100DE000A3E0FB7F02122DFE7E647F75906476E0A7
:100DF0002404FD122C6D906355E0F50A020A71E59A
:100E00000A64016003020A71906577E01460462469
:100E1000FE6042147003020EF224046003020A71A1
:100E2000E4F50C200F139065777404F0906575E07D
:100E30005401F0750A01020A719080027410F0E406
:100E4000906577F090657504F0750AFA9066827483
:100E5000FFF0020A71906682E07003020EDC90647B
:100E6000757480F09064777401F0E4A3F0A304F04B
:100E7000A37430F0A3747BF0E4F524747C2524F58E
:100E800082E43464F583747DF0747D2524F582E476
:100E90003464F583E4F0E5242407906476F07C66FE
:100EA0007D82906349E0FAA3E0FB7F02122DFE7E73
:100EB000647F75E5242409FD122C6D906681E06045
:100EC0001B1233FBD203E4F50A906575F090668639
:100ED00004F0E4906679F0A3F0020A71300F07E4A1
:100EE000906577F080069065777404F0750AFA02D1
:100EF0000A719080027410F0750A05906575E064BF
:100F000001FFF09065777401F0EF7019906351E084
:100F10006013FCA3E0FDA3E0FEA3E0FF9066821255
:100F20001AEE020A7190634DE0FCA3E0FDA3E0FE1F
:0E0F3000A3E0FF906682121AEE020A7180FEA4
:010F3E002290
:10002600906376E0B444047F0180027F009063759C
:10003600E0B447047E0180027E00EE5F604A906372
:100046003EE0906377F090633FE0906378F09063D2
:1000560040E0906379F0906341E090637AF09063BA
:1000660042E090637BF0906343E090637CF09063A2
:10007600767452F09062AE63A2019080A863A201EA
:100086007F06121D4D0208C6906331E0C3940850E6
:10009600030208CF90633EE0FF906377E06F600352
:1000A6000208CF90633FE0FF906378E06F60030241
:1000B60008CF906340E0FF906379E06F6003020829
:1000C600CF906341E0FF90637AE06F60030208CF50
:1000D600906342E0FF90637BE06F60030208CF907D
:1000E6006343E0FF90637CE06F60030208CF906398
:1000F60076E06444701A9080A8E0B4FF139062AE74
:1001060063A2019080A863A2017F06121D4D801094
:100116009062B2E09080ACF09062B3E09080ADF077
:1001260090668DE060037401F090668E7464F090C2
:1001360063767452F0906375E0646D600302026941
:100146007BFF7A0F796B1213FA7BFF7A0F79859012
:10015600633EE0F52DA3E0F52EA3E0F52FA3E0F531
:1001660030A3E0F531A3E0F5321213FA752DFF75D1
:100176002E0F752FE27530FF75310F7532EE7BFF4E
:100186007A0F79BB1213FA7BFF7A0F79F71213FAFB
:100196007BFF7A10795D1213FA7BFF7A10798A90C9
:1001A6006344E0F52DA3E0F52EA3E0F52FA3E0F5DB
:1001B600301213FA7BFF7A1079B490634DE0F52D77
:1001C600A3E0F52EA3E0F52FA3E0F5301213FA7B9A
:1001D600FF7A1079E2906351E0F52DA3E0F52EA3A6
:1001E600E0F52FA3E0F5301213FA7BFF7A117910B0
:1001F60090633AE0F52DA3E0F52EA3E0F52FA3E0FA
:10020600F5301213FA7BFF7A117933906336E0F5F5
:100216002DA3E0F52EA3E0F52FA3E0F5301213FA97
:100226007BFF7A1179501213FA7BFF7A117979A242
:100236000FE433F52D1213FA7BFF7A1179A9906634
:1002460081E0F52D1213FA7BFF7A1179D490668D31
:10025600E0F52D1213FA1231727BFF7A127907122A
:1002660013FA22906375E0644C70737E127F0DFB67
:10027600FDFC1222F790637DE0F525A3E0F526E468
:10028600F528E52590637FF0A3E526F07E127F48EA
:100296007C637D7F7B021222F7E4F5278526828523
:1002A6002583E0FF747F2527F582E43463F583EF29
:1002B600F00526E526700205250527E527B410DC9E
:1002C6007E127F4B7C637D7F7B101222F70528E52B
:1002D60028C3941040AC7E127F4E122502229063F2
:1002E60075E0646C7060F5297E127F50FBFDFC1290
:1002F60022F7E4F528E490637FF0A3E529F07E1267
:100306007F487C637D7F7B021222F7E4F527A829CC
:10031600E6FF747F2527F582E43463F583EFF00565
:10032600290527E527B410E67E127F4B7C637D7F87
:100336007B101222F70528E528C3940840B77E12E1
:100346007F4E12250222906375E0644B7061F5279B
:1003560074672527F582E43463F583E060327467B9
:100366002527F582E43463F583E0F460237467257A
:1003760027F582E43463F583E0FF747D2527F58253
:10038600E43463F583E0B507100527E527B408C014
:100396009061047432F00208C69063757421F030DF
:1003A6000B030208C67E127F8B1225020208C69036
:1003B6006375E0B4521A200B077E127F9312250252
:1003C6009063757472F07E637F757D08122BE6224A
:1003D600906375E064497045200B077E127F9E127C
:1003E600250290637DE0F525A3E0F526E4F5278553
:1003F6002682852583E0FF747F2527F582E4346312
:10040600F583EFF00526E526700205250527E52785
:10041600B480DC7E637F757D8A122BE6229063753D
:10042600E064437046200B077E127FA612250290D9
:10043600637DE0F525A3E0F526E4F527852682858C
:100446002583E493FF747F2527F582E43463F583DF
:10045600EFF00526E526700205250527E527B48079
:10046600DB7E637F757D8A122BE622906375E064DE
:100476005A7053200B077E127FAF12250290637DC0
:10048600E0F525A3E0F5267C637D7F7B80AF26AE75
:10049600251232A1E4F527852682852583E493FF7C
:1004A600747F2527F582E43463F583EFF00526E5AE
:1004B60026700205250527E527B480DB7E637F7558
:1004C6007D8A122BE622906375E064446003020580
:1004D6005D90637DE0FF644470030208C6EFB431AB
:1004E6000CC20B7E127FBB1225020208C690637DEA
:1004F600E0B4300CD20B7E127FC71225020208C66A
:1005060090637DE0B4320CD20C7E127FD4122502A9
:100516000208C690637DE0B4330CC20C7E127FE203
:100526001225020208C690637DE0B4340CD20D7E1B
:10053600127FF11225020208C690637DE0B4350CE5
:10054600C20D7E127FFE1225020208C690637DE070
:10055600FF1200210208C6906104E07013200B0709
:100566007E137F0C1225029063757421F00208C673
:100576009061047432F0906375E0FFB45104C2AF29
:1005860080FEEF64577045200B077E137F1A1225F5
:100596000290637EE0906331F0E4F527906331E0EA
:1005A600FFE527C39F40030208C6747F2527F5820F
:1005B600E43463F583E0FF90637DE0252724ADF501
:1005C60082E43461F583EFF0052780D0906375E00F
:1005D60064536003020680200B077E137F251225D5
:1005E6000290633EE0FF9061B6E06F703C90633F1F
:1005F600E0FF9061B7E06F7030906340E0FF90617C
:10060600B8E0B50724906341E0FF9061B9E0B50713
:1006160018906342E0FF9061BAE0B5070C9063431F
:10062600E0FF9061BBE06F60169063757421F03057
:100636000B030208C67E137F341225020208C6E4A5
:10064600F527E4F50DAF27FE74AD2527F582E434D2
:1006560061F583E0FD1233040527E527C394FE40C8
:10066600E1C2AFE4907FF0F0A3F0907FFD74AAF0B2
:10067600A374FFF0A37455F080FE906375E0644F99
:10068600705A90637DE0F525A3E0F526E52645251D
:10069600700A200B077E137F3D122502200B077E72
:1006A600137F44122502E4F527747F2527F582E49B
:1006B6003463F583E0852682852583F00526E526C5
:1006C600700205250527E527B480DE90668CE024B8
:1006D60080F090668BE03400F00208C6906375E007
:1006E6006445707490637DE0FEA3E0FF907FF0EEBA
:1006F600F0A3EFF0D39400EE94044038907FF0E03E
:10070600FEA3E0FF90668BE0FCA3E0FD9FEC9E401D
:1007160023E42FFFEE3401FED3ED9FEC9E5015C26D
:10072600AF907FFD74AAF0A374FFF0A37455F0E4B4
:10073600F5A780FE7E137F461225027BFF7A13798A
:100746004E907FF0E0F52DA3E0F52E90668BE0F558
:100756002FA3E0F5301213FA906375E06465600329
:100766000208CF90637DE0FFA3E0907FF0CFF0A377
:10077600EFF0E4F525F526D3907FF1E09526907FFE
:10078600F0E095254020E4F50D2526FFE52534010A
:10079600FE852682852583E0FD1233040526E5269F
:1007A6007002052580D17E137F59122CF4EF4E601E
:1007B60020120003906344EFF0120003906345EFAC
:1007C600F0120003906346EFF0120003906347EFC8
:1007D600F07E137F5F122CF4EF4E60201200039020
:1007E600634DEFF012000390634EEFF0120003909A
:1007F600634FEFF0120003906350EFF07E137F65B6
:10080600122CF4EF4E6020120003906351EFF012A9
:100816000003906352EFF0120003906353EFF0125F
:100826000003906354EFF07E137F6B122CF4EF4EAF
:10083600602012000390633AEFF012000390633BCE
:10084600EFF012000390633CEFF012000390633D5B
:10085600EFF07E137F71122CF4EF4E60201200032E
:10086600906336EFF0120003906337EFF012000347
:10087600906338EFF0120003906339EFF0E4F52748
:10088600E4F50DE5272401FFE433FE74362527F54C
:1008960082E43463F583E0FD1233040527E527C3BC
:1008A600944340DCC2AFE4907FF0F0A3F0907FFD6C
:1008B60074AAF0A374FFF0A37455F0E4F5A780FEC4
:0908C6007E637F757D08122BE6AC
:0108CF002206
:10326900AE07EEC39430400BEED394395005EE24EB
:10327900D0FF22EEC39461400BEED394665005EE65
:1032890024A9FF22EEC39441400BEED39446500586
:08329900EE24C9FF22AF06225A
:1033C6009062ADE004F070069062ACE004F09062AA
:0A33D600ACE0FEA3E0FF123370220A
:100003001233C6123269EFC454F0FEC0061233C66F
:08001300123269D0E02FFF2238
:10305F00E49068B3F01233C69068B4EFF0C39430C5
:10306F004018E0FFD3943950119068B3E02405F570
:10307F0082E43461F583EFF080119068B3E02405AA
:10308F00F582E43461F583E4F0800C9068B3E004DA
:10309F00F0E0D3940840BE752800752900752A000A
:0C30AF00E4F52B7B017A617905121E5BB1
:0130BB0022F2
:042CF4008E2A8F2B6A
:102CF8009062ACE4F0A374FFF01233C6EF606EF498
:102D0800606B852B82852A83E493B507EC752C01CB
:102D1800E52B252CF582E4352AF583E4936025908C
:102D280062ADE0252CFF9062ACE03400FE123370F7
:102D3800E52B252CF582E4352AF583E493B50704C1
:102D4800052C80CCE52B252CF582E4352AF583E487
:102D58009370A6E52C24FFFFE434FFFE9062ADE0FB
:102D68002FF09062ACE03EF07E007F0122E4FEFF8F
:012D78002238
:1026CB007E137F77122CF4EF4E70037F01227E1363
:1026DB007F7A122CF4EF4E600C1233C6EF24D02409
:1026EB00FF920F8002D20F7E137F80122CF4EF4EDD
:1026FB00600C1233C6EF24D0906681F08005E49015
:10270B006681F07E137F86122CF4EF4E600C123331
:10271B00C6EF24D090668DF08005E490668DF07E38
:10272B00137F8C122CF4EF4E600C1233C6EF24D0B7
:10273B0024FF92018002C20190633E63A201906666
:10274B007B63A2017F06121D4D30013B7E137F92EE
:10275B00122CF4EF4E603012000390667BEFF012F8
:10276B00000390667CEFF012000390667DEFF01291
:10277B00000390667EEFF012000390667FEFF0127D
:0A278B000003906680EFF07F00224B
:10322200906576E0C3947C503D906576E0FE04F0B4
:1032320074B42EF582E43462F583EFF0BF0A27906E
:103242006576E0FF04F074B42FF582E43462F5830E
:10325200E4F0906576E0FF122D799065767408F0BF
:073262009062B5E004F022C8
:103118009080007480F090633663A201F583F58295
:1031280063A2017F08121D4D90633E63A201908047
:103138008863A2017F0A121D4D9080927407F0A344
:1031480074D0F0A37406F0906348E0FF9080B1F06B
:103158009080E1EFF09080957455F0A3F090800096
:0A3168007401F090800974F0F02269
:102FF100908009E04410F09080A0E070609080A182
:103001007482F09080A874FFF0A3F0A3F0A3F07F86
:10301100039080AEEFF0A374CBF09080007402F0C7
:103021009068A7121AFA000000009068A7E090804B
:1030310040F09068A8E0908041F09068A9E090800D
:1030410042F09068AAE0908043F0A3E4F0A3F0A3DB
:0D305100F0A3F0908018F0A3F0A3F0A3F01E
:01305E00224F
:1030BC00908009E04440F09080D17482F07F0390BE
:1030CC0080DEEFF0A374CCF09080027402F0906874
:1030DC00AB121AFA000000009068ABE0908058F038
:1030EC009068ACE0908059F09068ADE090805AF018
:1030FC009068AEE090805BF0A3E4F0A3F0A3F0A3A3
:0B310C00F0908030F0A3F0A3F0A3F0DF
:013117002295
:102F0000908009E04420F09080B8E0706C9080B927
:102F10007482F07F039080C6EFF07FCDA3EFF07F47
:102F2000039080C4EFF0A374CDF09080C074FFF0E4
:102F3000A3F0A3F0A3F09080017402F09068AF12A8
:102F40001AFA000000009068AFE090804CF09068A2
:102F5000B0E090804DF09068B1E090804EF09068C5
:102F6000B2E090804FF0A3E4F0A3F0A3F0A3F090C0
:092F70008024F0A3F0A3F0A3F00B
:012F79002235
:102DFE008C258D26A907EAFDE975F018A424ACFFF1
:102E0E00E5F034808F82F583EDF0EBFDE975F01877
:102E1E00A4FFAEF024ACFBEE34808B82F583A3EDE1
:102E2E00F08526828C83E0FDEF24A8FFEE3480FE31
:102E3E008F82F583EDF08526828C83A3E08F828EC0
:102E4E0083A3F0852682852583A3A3E0FDE975F093
:102E5E0018A424A8FFE5F03480FE8F82F583A3A387
:102E6E00EDF08526828C83A3A3A3E08F828E83A3AD
:042E7E00A3A3F022F8
:062BE6008D2AAB07AA06D0
:102BEC00908000E030E5079065787401F0229068E1
:102BFC00A7E0FCA3E0FDA3E0FEA3E0F52E8E2D8D57
:102C0C002C8C2BAE02AF038E838F8263A201E52D39
:102C1C00540744C0F583852E8263A201AF2A121D8E
:102C2C00BFE4FCFDFEE52E252AF52EEE352DF52D07
:102C3C00ED352CF52CEC352BF52B908040E52BF05D
:102C4C00A3E52CF0A3E52DF0A3E52EF09080007405
:102C5C0020F0AF2EAE2DAD2CAC2B9068A7121AEE37
:012C6C002245
:062C6D008D25AB07AA064D
:102C7300908002E030E5079065787403F022906855
:102C8300ABE0FCA3E0FDA3E0FEA3E0F5298E288DD5
:102C9300278C26AE02AF038E838F8263A201E528C1
:102CA300540744D0F58385298263A201AF25121D01
:102CB300BFE4FCFDFEE5292525F529EE3528F52899
:102CC300ED3527F527EC3526F526908058E526F0D7
:102CD300A3E527F0A3E528F0A3E529F0908002748B
:102CE30020F0AF29AE28AD27AC269068AB121AEEC0
:012CF30022BE
:0228FD008F2525
:1028FF00908001E030E5099065787402F07F002246
:10290F009068AFE0FCA3E0FDA3E0FEA3E0F5298E05
:10291F00288D278C2690667B63A201E528540744F7
:10292F00C8F58385298263A2017F06121DD5E5298B
:10293F002406F529E43528F528E43527F527E4356D
:10294F0026F52690657963A201E528540744C8F55A
:10295F008385298263A201AF25121DD5E4FCFDFEFC
:10296F00E5292525F529EE3528F528ED3527F52715
:10297F00EC3526F52690804CE526F0A3E527F0A34D
:10298F00E528F0A3E529F09080017420F0AF29AE7F
:0D299F0028AD27AC269068AF121AEEAF25C8
:0129AC002208
:1023FE009081E0E0F5250525052505250525052512
:10240E0005250525052505250525908010E0F528CF
:10241E00A3E0F529A3E0F52AA3E0F52B9081E1E0F6
:10242E00F52505250525052505250525052505255E
:10243E00052505250525908014E0F52CA3E0F52D46
:10244E00A3E0F52EA3E0F52FE52EB52A08E52FB56E
:10245E002B037F0022E4F525E52E540744E0F58397
:10246E00852F8263A20190637563A2017F08121EFD
:10247E000590637763A2019062AE63A2017F06129C
:10248E001D4D906375E0F526A3E0F527E4F5259044
:10249E006375E0702AA3E024F8F525E52E54074471
:1024AE00E0F583852F8274082582F582E43583F565
:1024BE008363A20190637563A201AF25121E05AE60
:1024CE0026E4FCFDE52F2527F52FE52E3EF52EED16
:1024DE00352DF52DEC352CF52C908014E52CF0A334
:1024EE00E52DF0A3E52EF0A3E52FF09080007440CB
:0324FE00F0AF2517
:0125010022B7
:101FFF009081E6E0F525052505250525052505250F
:10200F0005250525052505250525908028E0F528BA
:10201F00A3E0F529A3E0F52AA3E0F52B9081E7E0F3
:10202F00F525052505250525052505250525052561
:10203F0005250525052590802CE0F52CA3E0F52D31
:10204F00A3E0F52EA3E0F52FE4F525E52EB52A0A3A
:10205F00E52FB52B05C20802216BE52E540744F07E
:10206F00F583852F8263A20190637563A2017F08B8
:10207F00121E05906375E0F526A3E0F527E52745C9
:10208F002670099080027410F07F0022906682E023
:10209F00FFF46030906377E06F6003022132906647
:1020AF0083E0FF906378E06F7079906684E0FF9033
:1020BF006379E06F706D906685E0FF90637AE06FF3
:1020CF006031805F906377E0906682F0906378E094
:1020DF00906683F0906379E0906684F090637AE085
:1020EF00906685F090637BE0FFA3E0906349CFF0AB
:1020FF00A3EFF0906375E0702AA3E024F8F525E5CF
:10210F002E540744F0F583852F8274082582F582BB
:10211F00E43583F58363A20190637563A201AF2554
:10212F00121E05AE26E4FCFDE52F2527F52FE52E23
:10213F003EF52EED352DF52DEC352CF52CAF2BAEC8
:10214F002AAD29AC28AB2FAA2EA92DA82CD3121A51
:10215F00DD40099080027410F07F002290802CE502
:10216F002CF0A3E52DF0A3E52EF0A3E52FF0908042
:06217F00027440F0AF25E0
:012185002237
:102186009081E3E0F5250525052505250525052589
:102196000525052505250525052590801CE0F5283E
:1021A600A3E0F529A3E0F52AA3E0F52B9081E4E06E
:1021B600F5250525052505250525052505250525D9
:1021C600052505250525908020E0F52CA3E0F52DB5
:1021D600A3E0F52EA3E0F52FE4F525E52EB52A0AB2
:1021E600E52FB52B05C2090222DCE52E540744E88B
:1021F600F583852F8263A20190600463A2017F0E9E
:10220600121E1B906004E0F526A3E0F52790600CF3
:10221600E0FFF4604A90667BE0FEEF6E7079A3E023
:10222600FF90600DE06F706F90667DE0FF90600E2E
:10223600E06F706390667EE0FF90600FE06F70570E
:1022460090667FE0FF906010E06F704B906680E0D4
:10225600FF906011E06F703FE4906013F08008908B
:10226600601374FFF0D2D9906004E0702AA3E024D2
:10227600F2F525E52E540744E8F583852F82740E82
:102286002582F582E43583F58363A20190600463B9
:10229600A201AF25121E1BAE26E4FCFDE52F252765
:1022A600F52FE52E3EF52EED352DF52DEC352CF5DD
:1022B6002CAF2BAE2AAD29AC28AB2FAA2EA92DA860
:1022C6002CD3121ADD5006E52745267009908001A9
:1022D6007410F07F0022908020E52CF0A3E52DF00D
:1022E600A3E52EF0A3E52FF09080017440F0AF2512
:0122F60022C5
:042502008E2A8F2B63
:10250600908000E030E5079065787401F0229068CD
:10251600A7E0FCA3E0FDA3E0FEA3E0F5318E308D3D
:102526002F8C2EE531FFE5305407FEE42FF52DEE16
:1025360034C0F52C852D82F5837423F0052DE52D09
:102546007002052C532CC7F582852C83740AF0057E
:102556002DE52D7002052C532CC790633E63A20116
:10256600852C83852D8263A2017F06121DBF74060A
:10257600252DF52DE4352CF52C852A83852B8263B4
:10258600A201852C83852D8263A201121DA3E4FC82
:10259600FDFE9068A7E0F8A3E0F9A3E0FAA3E02F18
:1025A600FFEE3AFEED39FDEC38FCEF2408FFE43E81
:1025B600FEE43DFDE43CFC9068A7121AEE9068A785
:1025C600E0908040F09068A8E0908041F09068A983
:1025D600E0908042F09068AAE0908043F0908000FE
:0325E6007420F06E
:0125E90022CF
:0A22F7008E2A8F2B8C2C8D2D8B2E40
:10230100908000E030E5079065787401F0229068D4
:10231100A7E0FCA3E0FDA3E0FEA3E0F5348E338D3E
:10232100328C31E534FFE5335407FEE42FF530EE0E
:1023310034C0F52F853082F5837423F00530E53004
:102341007002052F532FC7F582852F83740AF0057C
:1023510030E5307002052F532FC790633E63A20111
:10236100852F8385308263A2017F06121DBF74060B
:102371002530F530E4352FF52F852A83852B8263AF
:10238100A201852F8385308263A201121DA38F359F
:10239100EF2530F530E4352FF52FE52E6017852C2C
:1023A10083852D8263A201852F8385308263A201FB
:1023B100AF2E121DBFE5352408252EF52EFFE4FCB6
:1023C100FDFEE5342FF534EE3533F533ED3532F5D9
:1023D10032EC3531F531908040E531F0A3E532F052
:1023E100A3E533F0A3E534F09080007420F0AF341E
:0C23F100AE33AD32AC319068A7121AEE8A
:0123FD0022BD
:022D79008F3E8B
:102D7B00908000E030E5079065787401F022906850
:102D8B00A7E0FCA3E0FDA3E0FEA3E0F5428E418D9E
:102D9B00408C3FE542FFE5415407FEE42FFFEE3444
:102DAB00C09062B463A201F5838F8263A201AF3E30
:102DBB00121DBFE4FCFDFEE542253EF542EE35411A
:102DCB00F541ED3540F540EC353FF53F908040E562
:102DDB003FF0A3E540F0A3E541F0A3E542F090807E
:102DEB00007420F0AF42AE41AD40AC3F9068A712EB
:022DFB001AEECE
:012DFD0022B3
:0625EA008E258F26AB05D3
:1025F000908000E030E5079065787401F0229068E3
:10260000A7E0FCA3E0FDA3E0FEA3E0F52C8E2B8D5C
:102610002A8C29E52CFFE52B5407FEE42FF528EE44
:1026200034C0F527852882F5837423F00528E52832
:10263000700205275327C7F582852783EBF005280D
:10264000E5287002052790633E63A20185278385F4
:10265000288263A2017F06121DBF74062528F52873
:10266000E43527F5275327C7E52585288285278365
:10267000F00528E528700205275327C7F58285272E
:1026800083E526F00528E528700205275327C7E5CE
:102690002C240AF52CE4352BF52BE4352AF52AE415
:1026A0003529F529908040E529F0A3E52AF0A3E536
:1026B0002BF0A3E52CF09080007420F0AF2CAE2B13
:0A26C000AD2AAC299068A7121AEEAB
:0126CA0022ED
:10337000A2AF9210C2AF438E2075D2028F828E838D
:0C338000E0FFE4F5D2538EDFA21092AF04
:01338C00221E
:10330400E5D220E0FBA2AF9210C2AF43D2028F827B
:103314008E83EDF075D25063D250A21092AFE5D2F5
:0333240020E0FBAB
:013327002283
:102E8200E4FDED2401FFE433FE12337074362DF5B8
:102E920082E43463F583EFF00DBD3FE6E4FDED24FB
:102EA2007FFFE433FE123370742D2DF582E434611A
:102EB200F583EFF0742D2DF582E43461F583E07033
:102EC2001B742D2DF582E43461F5837420F0742E89
:102ED2002DF582E43461F583E4F080040DBD80BEFB
:102EE200E49061ACF0FDEDFF7E0012337074AD2D05
:0D2EF200F582E43461F583EFF00DBDFEE9DB
:012EFF0022B0
:0232A1008B2A76
:1032A300A2AF9210C2AF85A22B53A2FE8E838F8250
:1032B30005A28C838D827409121E49E52A53A2FE4E
:1032C30043A220121E4B53A2DF852BA2A21092AF62
:0132D300FFFB
:0132D40022D7
:10338D00A2AF9210C2AF8C838D82EF121E4943A261
:0C339D0020121E4B53A2DFA21092AFFFC3
:0133A9002201
:023328008F25EF
:10332A00A2AF9210C2AFE4F5838D827406121E49D1
:10333A00E52543A220121E4B53A2DFA21092AF7FB3
:01334A000181
:01334B00225F
:02334C008F25CB
:10334E00A2AF9210C2AFE4F5838D82740A121E49A9
:10335E00E52543A220121E4B53A2DFA21092AF7F8F
:01336E00015D
:01336F00223B
:101C7200A907E7FFA805EF93C3966008403B74FCF1
:101C82002FFF80F00F08EF93C3966008402B74FB80
:101C92002FFF80E00F08EF93C3966008401B74FA91
:101CA2002FFF80D00F08EF93D3966008400B74F992
:101CB2002FFF80C01F1F1F1F1FEF54FEF80303F7E3
:101CC200E893FC08E893FD08E893FE08E893FF22F6
:101CD20009E993C39D6008402974FB29F980F10941
:101CE200E993C39E6008401A74FA29F980E209E96F
:101CF20093D39F6008400B74F929F980D3191919FD
:101D02001919E9C313C313FF22740093F8ECC398A3
:101D12004024701F740193F8EDC398401970147435
:0E1D22000293F8EEC398400E7009740393F814
:101D3000EFC39840037F00227F0122EDF8E6F00810
:101D4000A3DFFA22EDF8E0F608A3DFFA22E0A363AE
:101D5000A201F0A363A201DFF475A2002263A20135
:101D6000F0A363A20122E0A363A201F0A363A20196
:101D7000E0A363A201F0A363A201E463A201F0A3C4
:101D800063A201DFE175A20022E0A363A2016DFE60
:101D9000936CFDEE058393FC158363A201DFEA7566
:101DA000A200227F00E493A363A201F00F600CA3C2
:101DB000E583C2E3F58363A20180EA75A20022E015
:101DC000A363A201F0A3E583C2E3F58363A201DF6D
:101DD000EE75A20022E0A363A201F0A3E583C2E4B2
:101DE000D2E3F58363A201DFEC75A20022E0A363D6
:101DF000A201F0A3E58344F8C2E5F58363A201DF05
:101E0000EC75A20022E583C2E3F583E0A363A2019F
:101E1000F0A363A201DFEE75A20022E583C2E4D243
:0A1E2000E3F583E0A363A201F0A341
:101E2A0063A201DFEC75A20022E58344F8F583E0A2
:101E3A00A363A201F0A363A201DFEE75A20022F957
:101E4A0022C002C004C00612FFF0D006D004D0029D
:011E5A002265
:1016F4003E2A2C312CCFE0F0E0ECE5F2F0FB20ECBC
:10170400E0E3E8F1F2F0E0EBFCEDEEE3EE20EFEEE7
:10171400F0F2E00A003E4C2C4930312C256C752C3B
:10172400D1EAEEF0EEF1F2FC20EEE1ECE5EDE02C96
:1017340035302C3130302C3330302C3630302C31A5
:101744003230302C323430302C343830302C39367E
:1017540030302C31393230302C33383430302C3571
:10176400373630302C3131353230300A003E532C8C
:101774004930332C2562752CC7E0E4E5F0E6EAE055
:1017840020F1F2E0F0F2E020EFE5F0E5E4E0F7E844
:10179400282A3130ECF1290A003E532C4930342CEC
:1017A4002562752CCFE0F3E7E020EFE5F0E5E4E017
:1017B400F7E820EFE0EAE5F2EEE2282A3130ECF136
:1017C400290A003C21003C4930313D003C4930337A
:1017D4003D003C4930343D000AC1F3F4E5F020E714
:1017E400E0EDFFF221000A4F55543E000A3C002070
:1017F400212121435243204552523A2000008912AC
:101804009B24AD36BF48C15AD36CE57EF78108935B
:101814001AA52CB73EC940DB52ED64FF76028B104B
:101824009926AF34BD4AC358D16EE77CF5830A913B
:1018340018A72EB53CCB42D950EF66FD74048D1623
:101844009F20A932BB4CC55ED768E17AF3850C971B
:101854001EA128B33ACD44DF56E960FB72068F140B
:101864009D22AB30B94EC75CD56AE378F1870E95FB
:101874001CA32AB138CF46DD54EB62F97008811AF3
:10188400932CA53EB740C952DB64ED76FF89009BDB
:1018940012AD24BF36C148D35AE56CF77E0A8318CB
:1018A400912EA73CB542CB50D966EF74FD8B0299BB
:1018B40010AF26BD34C34AD158E76EF57C0C851EA3
:1018C4009728A13AB344CD56DF60E972FB8D049F9B
:1018D40016A920BB32C54CD75EE168F37A0E871C8B
:1018E400952AA338B146CF54DD62EB70F98F069D7B
:1018F40014AB22B930C74ED55CE36AF178001123EA
:1019040032465765748C9DAFBECADBE9F8100133CB
:1019140022564775649C8DBFAEDACBF9E8213002BC
:101924001367764455ADBC8E9FEBFAC8D9312012AB
:101934000377665445BDAC9E8FFBEAD8C942536118
:101944007004152736CEDFEDFC8899ABBA5243718B
:101954006014053726DECFFDEC9889BBAA6372407C
:101964005125340617EFFECCDDA9B88A9B7362506B
:101974004135241607FFEEDCCDB9A89A8B8495A7D0
:10198400B6C2D3E1F008192B3A4E5F6D7C9485B74B
:10199400A6D2C3F1E018093B2A5E4F7D6CA5B4863C
:1019A40097E3F2C0D129380A1B6F7E4C5DB5A4962B
:1019B40087F3E2D0C139281A0B7F6E5C4DC6D7E598
:1019C400F48091A3B24A5B69780C1D2F3ED6C7F50B
:1019D400E49081B3A25A4B79681C0D3F2EE7F6C4FC
:1019E400D5A1B082936B7A48592D3C0E1FF7E6D4EB
:0D19F400C5B1A092837B6A58493D2C1E0F9F
:1033B00052668F00000000000000000000000000C6
:0533C000000000000008
:0100210022BC
:03002300022ACCE2
:0B2ACC00C0E0C083C082C0D075D018ED
:102AD70030984BC298750B01AF99E543700EEF64C0
:102AE70055703BF54A754301D2918032E553702EFC
:102AF70074A1254AF582E43466F583EFF0E54AB41C
:102B07000104EF04F544E54A600AB5440F04F553A0
:102B1700C2918008EF64556003754300054A3099F8
:102B270029301A24D290E551B5490DC21AD21CC2D8
:102B370090D296854508801074A12551F582E4341A
:0A2B470067F583E0F5990551C29986
:092B5100D0D0D082D083D0E03254
:103172007BFF7A1679F41213FA9068A1E0FEA3E0BD
:10318200FFC3E49FFFE49EFEAB07FA3395E0F9F834
:103192007F007E8C7D0A7C00121A3D8F308E2F8D2F
:1031A2002E8C2D7BFF7A1779191213FA7BFF7A176F
:1031B2007971E54614F52D1213FA7BFF7A17799D82
:0931C200E54514F52D1213FA2263
:102F7A007E177FC7122CF4EF4E70037F01227E1753
:102F8A007FCA122CF4EF4E602312305FA804A90501
:102F9A00AA06AB077F007E8C7D0A7C00121A3D12BE
:102FAA001ACF9068A1EEF0A3EFF0800A9068A1749E
:102FBA00FFF0A374B8F07E177FD0122CF4EF4E60A6
:102FCA000912305FEF04F5468003E4F5467E177F69
:102FDA00D6122CF4EF4E600912305FEF04F54580EB
:072FEA0003E4F5457F00221E
:1031CB00C21AC21CE4F543F551F549F54AF50BC299
:1031DB0019755209122F7AD296C2ADE4F5C9D2CD28
:1031EB00D2CCC2C9C2CAF5CDF5CC9068A1E0F5CB63
:1031FB00A3E0F5CA85CBCD85CACCE4F598D29E4326
:10320B008740C29FC2ACC298C29975B81075B710EF
:07321B00D2CAD29CD2AC2202
:0100220022BB
:10279500E4FF0F2405F582E43461F583E552F00F7B
:1027A50074052401F582E43461F583E4F07C667DEB
:1027B50094FEED1DAA0470011CF5828A83E0FBAA34
:1027C500070F74052AF582E43461F583EBF00EBE3C
:1027D50004E07C667D98E4FEED1DAA0470011CF5FD
:1027E500828A83E0FBAA070F74052AF582E4346127
:1027F500F583EBF00EBE04E07C667D9CE4FEED1DEA
:10280500AA0470011CF5828A83E0FBAA070F7405F0
:102815002AF582E43461F583EBF00EBE04E07C66B4
:102825007DA0E4FEED1DAA0470011CF5828A83E0FB
:10283500FBAA070F74052AF582E43461F583EBF0F2
:042845000EBE04E0DF
:01284900226C
:03001E00D2992252
:0733FB00D2CAD29CD2AC2221
:10284A008F25301A0E300B030228FC7E177FDC120C
:10285A00250222906378E0F5527F797583630582B9
:10286A0063A2019067A463A201E52524FCFF121D5F
:10287A004D9067A17455F0A3F0E52524FEA3F0E579
:10288A002504F549E4F54DF54EE52524FCF5507F80
:10289A00A4758367058263A20190180163A201AF40
:1028AA0050AE4FAD4EAC4D121D898F508E4F8D4E8E
:1028BA008C4D749F2549F582E43467F583E54EF023
:1028CA0074A02549F582E43467F583E54DF0E4F513
:1028DA0051D21AC296E5462508F508700312001E61
:1028EA00200B0D7E177FEA7C677DA1AB491222F788
:0328FA00C21C22DB
:102A3D00E5537002FF22E55324FEF5259066A3634E
:102A4D00A20190647963A201AF25121D4DE4F543F7
:102A5D00F553906475F0E52524FEA3F090667AE0B9
:102A6D00906477F0A37419F0E4F54DF54E8525507B
:102A7D007F79758364058263A20190180163A201B9
:102A8D00AF50AE4FAD4EAC4D121D898F508E4F8D48
:102A9D004E8C4D200B0D7E177FF07C647D79AB2520
:102AAD001222F7E54E454D6013200B0D7E177FF377
:0E2ABD007C007D4D7B021222F77F00227F01FC
:012ACB0022E8
:0134020022A7
:1032D500300004C2000547300E04C20E054BE50858
:1032E500B40109E4F508301A0312001E301A0CE582
:0F32F50047D394144008C21AD21C22E4F5472292
:0B33F000301C05C21C7F01227F002260
:102B66000208D0E493A3F8E493A34003F68001F2AD
:102B760008DFF48029E493A3F85407240CC8C33370
:102B8600C4540F4420C8834004F456800146F6DF3F
:102B9600E4800B01020408102040809033AAE47EF2
:102BA600019360BCA3FF543F30E509541FFEE49334
:102BB600A360010ECF54C025E060A840B8E493A3FB
:102BC600FAE493A3F8E493A3C8C582C8CAC583CA26
:102BD600F0A3C8C582C8CAC583CADFE9DEE780BEDE
:0133C5000007
:101A010075F008758200EF2FFFEE33FECD33CDCC9C
:101A110033CCC58233C5829BED9AEC99E58298401F
:101A21000CF582EE9BFEED9AFDEC99FC0FD5F0D6FC
:101A3100E4CEFBE4CDFAE4CCF9A88222B800C1B926
:101A41000059BA002DEC8BF084CFCECDFCE5F0CB64
:101A5100F97818EF2FFFEE33FEED33FDEC33FCEB9D
:101A610033FB10D703994004EB99FB0FD8E5E4F958
:101A7100FA227818EF2FFFEE33FEED33FDEC33FC45
:101A8100C933C910D7059BE99A4007EC9BFCE99A39
:101A9100F90FD8E0E4C9FAE4CCFB2275F010EF2F7E
:101AA100FFEE33FEED33FDCC33CCC833C810D7077E
:101AB1009BEC9AE899400AED9BFDEC9AFCE899F8B9
:0E1AC1000FD5F0DAE4CDFBE4CCFAE4C8F9224C
:0E1ACF00C3E49FFFE49EFEE49DFDE49CFC2228
:101ADD00EB9FF5F0EA9E42F0E99D42F0E89C45F05F
:011AED0022D6
:0C1AEE00ECF0A3EDF0A3EEF0A3EFF0226B
:101AFA00A8828583F0D083D082121B11121B111287
:101B0A001B11121B11E473E493A3C583C5F0C583AB
:101B1A00C8C582C8F0A3C583C5F0C583C8C582C835
:011B2A002298
:10139800E539242DF8E6053922782A301702782D08
:1013A800E475F001121BD2021B2B2010EB7F2ED20A
:1013B800108018EF540F2490D43440D4FF30140B0D
:1013C800EF24BFB41A0050032461FFE53A60021508
:1013D8003A053DE53D7002053C30170D782AE47565
:1013E800F001121BD2EF021B710232227403D217D2
:1013F8008003E4C217F5398B2A8A2B892CE4F53A45
:10140800F53CF53DE53A60077F201213D380F5756A
:101418003BFFC211C210C212C213C215C216C218B3
:101428001213A1FF700D3017057F001213E4AF3DB2
:10143800AE3C22B4255FC2D5C2141213A1FF24D03A
:10144800B40A00501A75F00A783A30D50508B6FF84
:101458000106C6A426F620D5047002D21380D9242A
:10146800CFB41A00EF5004C2E5D2140215E4D21129
:1014780080C6D21080C0D21280BCD2D580BAD21514
:1014880080B47F201213D32012077401B53A0040AC
:10149800F1121398FF1213D302140CD218D216802B
:1014A80095121398FB121398FA121398F94A4B7075
:1014B8000679B57A167BFF20122EE53A602A7E005F
:1014C8008E82758300121B4460060EEE653B70F039
:1014D800C2D5EBC0E0EAC0E0E9C0E0EE12162BD0BE
:1014E800E0F9D0E0FAD0E0FB121B2BFF60AAEBC0BA
:1014F800E0EAC0E0E9C0E01213D3D0E02401F9D05B
:10150800E03400FAD0E0FBE53B0460DCD53BD98051
:10151800877BFF7A167927D212809C79108002790E
:1015280008C216C2188008D2D5790A8004790AC27E
:10153800D5E53B047002F53BE4FAFDFEFF12139873
:10154800FC7B08201113121398FD7B1030100A122F
:101558001398FE121398FF7B20EC3382D592D55056
:1015680013C3E43010069FFFE49EFEE42011039DA0
:10157800FDE49CFCE4CBF8C211EC700CCFCECDCCD2
:10158800E824F8F870F38017C3EF33FFEE33FEED6D
:1015980033FDEC33FCEB33FB994002FB0FD8E9EB4E
:1015A800301105F8D0E0C448B211C0E00AEC4D4E45
:1015B8004F78207B0070C2EAB53B0040BCC0E01207
:1015C800162DD0F0D0E0201104C4C0E0C4B211C080
:1015D800F01213BCD0F0D5F0EB02140C121C31142D
:1015E800A953152358147A4C14764215274F152FF2
:0F15F80044152F49148F431535551519461519EC
:101607004515194716D550147E2D14822E14A52B77
:1016170014862314A32016BE2A143E480000149DE6
:101627003F3F3F00790AA2D5201314301509B9109E
:10163700020404B9080104A2D520160250010420AF
:1016470012689212B53A005034C0E07F2030131967
:101657007F30A21272167215500F121684C212C270
:1016670016C215C2187F30800F301503E9C0E0128B
:1016770013D3301503D0E0F9D0E0B53ACC301517C5
:101687007F30B9100C1213D37F583014077F78803E
:1016970003B908031213D33012057F2D0213D37F2A
:1016A700202018F87F2B2016F322921280CF286E65
:1016B700756C6C2900D2111213983011F8C2117889
:1016C7003A30D50108F602143E2D504349581213FB
:1016D700982403B405004001E49016D0931213C474
:0D16E700743A1213C4D213753A040215238D
:101E5B008B258A268927E4F531F530F52FF52EF5FC
:101E6B002CF52DE529452A45286012EBC0E0EAC088
:101E7B00E0E9C0E0AB28AA29A92A121BE2AB250591
:101E8B0027E527AA267002052614F9121B2BF5321B
:101E9B00C394094007E532D3940D40E1E532642049
:101EAB0060DBE532B42D05432D038016E532B42BF0
:101EBB0005432D01800C74FF2527F52774FF35266C
:101ECB00F526E52B60046410703FAB25AA26A927E5
:101EDB00121B2B64306009E52B702E752B0A8029A1
:101EEB00900001121B44FF64786004EFB458134355
:101EFB002D01752B1074022527F527E43526F526C1
:101F0B008007E52B7003752B08AB250527E527AA62
:101F1B00267002052614F9121B2BF532C39461406F
:101F2B000AE532D3947A50035332DF74D02532F55D
:101F3B0032C3940A400CE5329411406D74F925328A
:101F4B00F532E532D3952B5060432D018531368523
:101F5B003035852F34852E33AF2B7E00E4FCFDAB63
:101F6B0031AA30A92FA82E121B83C8ECC8C9EDC902
:101F7B00CAEECACBEFCBE4FCFDFEEB2532F531EE1E
:101F8B003AF530ED39F52FEC38F52EAF31AE30ADEB
:101F9B002FFCAB36AA35A934A833D3121ADD500364
:101FAB00021F14432D04021F14E52D20E003E480CF
:101FBB002DE529452A4528601EAB25E52724FFF989
:101FCB00E52634FFFAEBC0E0EAC0E0E9C0E0AB285D
:101FDB00AA29A92A121BE2E52D30E20774FFFFFEA6
:101FEB00FDFC22E52DAF31AE30AD2FAC2E30E10331
:041FFB00021ACF22D5
:101B2B00BB010689828A83E0225002E722BBFE02B8
:091B3B00E32289828A83E49322EB
:101B4400BB010CE58229F582E5833AF583E0225056
:101B540006E92582F8E622BBFE06E92582F8E222A0
:0D1B6400E58229F582E5833AF583E49322BA
:101B7100BB010689828A83F0225002F722BBFE0153
:021B8100F3224D
:101B8300E88FF0A4CC8BF0A42CFCE98EF0A42CFC01
:101B93008AF0EDA42CFCEA8EF0A4CDA8F08BF0A47F
:101BA3002DCC3825F0FDE98FF0A42CCD35F0FCEBDE
:101BB3008EF0A4FEA9F0EB8FF0A4CFC5F02ECD39A3
:0F1BC300FEE43CFCEAA42DCE35F0FDE43CFC2210
:101BD200FAE6FB0808E6F925F0F618E6CA3AF62214
:101BE200BB011A89828A83D0F0D0E0F8D0E0F9D024
:101BF200E0FAD0E0FBE8C0E0C0F0021C605016E959
:101C0200F8D083D082D0E0F9D0E0FAD0E0FBC082F5
:101C1200C083021C57BBFE16E9F8D083D082D0E005
:0F1C2200F9D0E0FAD0E0FBC082C083021C692237
:101C3100D083D082F8E4937012740193700DA3A342
:101C410093F8740193F5828883E473740293686056
:061C5100EFA3A3A380DF56
:091C5700EBF608EAF608E9F622B2
:091C6000EBF0A3EAF0A3E9F02285
:091C6900EBF208EAF208E9F222AC
:00000001FF
